:1000000028F107208D0200009102000093020000F9
:1000100095020000970200009902000062FFF7DFDE
:100020000000000000000000000000009B02000033
:100030009D020000000000009F0200007B250000E0
:10004000A3020000A3020000A3020000A30200001C
:10005000A3020000A3020000A3020000A30200000C
:10006000A3020000A3020000A3020000A3020000FC
:10007000A3020000A3020000A3020000A3020000EC
:10008000A3020000A3020000A3020000A3020000DC
:10009000A3020000A3020000A3020000A3020000CC
:1000A0009F1C0000A3020000A3020000A3020000A6
:1000B000A3020000A3020000A3020000A3020000AC
:1000C000A3020000A3020000A3020000DFF80CD08E
:1000D00004F01EFC004800472109000028F1072019
:1000E000D0F800D0D0F804F070B500230E4D0AE02F
:1000F000CE5C04885B1C86EA14269BB235F8166039
:1001000086EA04240480521E92B2F1D270BD30B54A
:10011000064C0022855CA35C521C1D4492B2CD5457
:10012000FF2AF7D930BD0000F84C0000F84B000062
:100130004F4A104710B572B633244E4B10C307C355
:100140004D484FF47A710068B0FBF1F01860191D4A
:100150004848FFF7EDFF62B610BD464A32231360F0
:10016000C2E9010144484FF47A710068B0FBF1F034
:10017000D06002F114011046DAE73E4A34231360DE
:10018000C2E901013C484FF47A710068B0FBF1F01C
:10019000D06002F114011046CAE710B572B6062409
:1001A000364900BF51F82420824212D933497839A8
:1001B00051F82410814207D121460846FFF7CDFFB0
:1001C00021460846FFF7D9FF21460846FFF7C5FF3D
:1001D00002E0641C1D2CE5D962B610BD2DE9F0418A
:1001E000274C236803B92060224D0020283563681E
:1001F00003E00F5C1E18401CAF559042F9D39818CD
:100200004FF480766060B04213D12068FFF7C5FFDD
:10021000184D1435286800B1FEE7164932462831DA
:100220002068FFF787FF286800B1FEE700206060C4
:1002300020600020BDE8F08172B61249124A0140E8
:100240001160FFF74DBF46F2044000210088A0F581
:100250001942993A0AD04FF4C0404FF4002208C81E
:1002600090421944FBD309B1002070470120704728
:10027000F11FFF1FBCDF072004C10720B04F0000A3
:10028000C4C0072080FFFF1F08ED00E005480047BD
:10029000FEE7FEE7FEE7FEE7FEE7FEE7FEE7FEE736
:1002A000FEE7FEE7CD000000EFF3108010F0010F35
:1002B00072B64FF080404FF0000202704FF0AA0378
:1002C00003724FF05504047202614FF0FF02426066
:1002D0004FF0030202700372047200D162B6FEE7AF
:1002E00010B50B4604461146184604F0FDFAC4E961
:1002F000000110BD7047000000000000FFFFFFFF7D
:1003000070B5224C2078002813D0214D012811D03F
:1003100002280ED1A8686168401A1E49884208D395
:100320001D48406B400004D5012001F092FB0020E5
:10033000207070BDA8686168401A18498842F8D3D7
:10034000002001F086FBA86860600220F0E700282A
:1003500002D10E4901200870704710B501F096F8DF
:100360000A490020087010BD0848012101700849A1
:1003700089684160704770477047022803D003289E
:1003800003D100F03EBE00F059BE7047F0C0072018
:1003900000000940A086010000C0092040420F0073
:1003A00040EA01039B0703D009E008C9121F08C0F7
:1003B000042AFAD203E011F8013B00F8013B521E77
:1003C000F9D2704730B50B460146002020220124A7
:1003D00009E021FA02F59D4205D303FA02F5491B13
:1003E00004FA02F52844151EA2F10102F1DC30BD29
:1003F00002E008C8121F08C1002AFAD170470000A5
:10040000000000008C0C000010B5FC49486D800411
:100410000CD4FB4A906843F698239468241A9C42B3
:10042000FBD3486D800401D4012010BD052001F0EC
:1004300033FD002010BD70B5F14CA668042001F01A
:100440002BFDF04D03E000BFFFF7DEFF48B1A068D1
:10045000801BA842F8D308E0FFF7D6FF08B10120BF
:1004600070BDA068801BA842F6D3002070BD2DE9A6
:10047000F041092001F010FDE34800264FF47A779F
:100480000670C821384601F0CBFEDD4CA06842F270
:100490001075A168091AA942FBD3C821384601F09A
:1004A000BFFEA068A168091AA942FBD3C82138463B
:1004B00001F0B6FED548022186708171C670BDE894
:1004C000F0814FF000098CB04620CDF828908DF8CF
:1004D00014008DF817904B20CA460090CDF8249058
:1004E0005446CBA3CBA20A2105A804F023FADFF8D7
:1004F0002CB3DBF800004FF6FF021040C84A40F46E
:1005000080701043CBF80000C648C849CA4D04604B
:10051000C5480068A0F56C50FF380860C44900F574
:10052000E0500860C349400A0860F8202870FF20A6
:100530006870A87001F00CFEB44CC049002094F91A
:10054000052051F822102A1802F580520B5C401C3D
:1005500082F800386028F6D34FF4E175294640F25E
:10056000491001F05DFE294640F29F1001F058FE4F
:100570004FF40055207808B1FFF7C2FEA07938B1DA
:10058000012819D003287DD0207800287BD08AE16B
:100590000A2001F081FC00F08BFE002874D10120BC
:1005A000A0714FF4005584F803A0062001F074FCFC
:1005B0000A2001F071FC8AE119222946A04800F0C6
:1005C00037FE9F48007E002876D09D480078062898
:1005D00071D2DFE800F0C3030B72727540F2044081
:1005E0009749008804904968814264D094484FF04C
:1005F0000109417A01295ED1D0F80A1019B991494F
:100600008969C0F80A108E484FF00006007A40074A
:1006100020D54FF480788A4F17E0072001F03CFC8A
:10062000A91942468848193100F002FE84498648DB
:100630001931FFF76CFDD7F80A0081493044424672
:100640001931FFF7CBFD06F58076D7F80E00B042E2
:10065000E3D823E0DFF8E8811BE0072001F01CFC71
:10066000D7F80E00B846871B402F00D94027A9199C
:100670003A467548193100F0DBFDD8F80A003A46D1
:10068000304402E0F6E007E1F1E06F49FFF7A6FD34
:100690003E44D8F80E004746B042DED8684801789C
:1006A00001295BD14FF0E0220906C2F88011D0F891
:1006B0000A00FFF7C1FD51E071E04FF0010950E081
:1006C0005F484FF00109417A03294AD156495F4AF0
:1006D0004FF000060B681360027A520720D54FF4E2
:1006E0008077804617E0072001F0D6FBA9193A462B
:1006F0005548193100F09CFD514953481931FFF715
:1007000006FD49483A46006881194D48193000F005
:100710007EFD06F58076D8F80E00B042E3D81DE0E5
:10072000804616E0072001F0B7FBD7F80E00871BC4
:10073000402F00D94027A9193A464348193100F003
:1007400077FD39483A46006881193F4800F05FFD5F
:100750003E44D8F80E004746B042E3D83848007E01
:10076000E8B1374E307AC00614D538494FF40050FE
:100770000122086005F1180104A8CDF810A000F0CE
:1007800037FD307820B1C8214FF47A7001F048FD70
:10079000307E20B1307A800701D5FFF785FD2848EB
:1007A0001B35D0F80E000544254800F075FD18B340
:1007B00002201549A0714FF4005581F800A00B20CC
:1007C00001F06AFBB9F1000F46D00D484FF0000967
:1007D000826842F210738168891A9942FBD34FF400
:1007E0002F714FF47A7001F01BFD0448406D4005F5
:1007F0002ED500200B902DE02EE0000000C0092037
:100800000000094080841E0068C00720BCC007208B
:100810004600000025732564000000000CED00E098
:100820000000FA05ACC00720B8C007209CC0072014
:1008300094C0072098C0072041C2072060C007204D
:1008400028C10720384F0000B9DC0720B0C00720BE
:100850000B9808B9FFF728FDE078401CC0B2E070A3
:100860000C2802D30120A07001E0A07878B3FFF734
:10087000FEFD2CE04B4881680A98091A099800EBA4
:100880004002C2EBC010B1EBC00F20D300200A9091
:10089000099084F806A01AE00120207001F018F9F0
:1008A000012001F0D6F84048007880B1002105A869
:1008B00000F010FC58B10320A0713A4884F803A05E
:1008C0004FF4005580680A904FF47A700990374EC3
:1008D000706D00053FF54EAE32488168344A83683A
:1008E0005B1A9342FBD3706D0005F3D4706D000565
:1008F000FCD44FF48040B06332214FF47A7001F0A1
:100900008FFC706DC0040AD5DBF80010294A01F491
:10091000E0611143CBF80010BFF34F8FFEE7FEE715
:10092000254C0025FF202560A580A571607101F090
:1009300061FB01F0A3FC01F010FE01F031FA002090
:1009400001F0AAFA01F032FE1848406DC0040CD53F
:10095000FFF75AFD48B1FFF76EFD30B1FFF76BFDB1
:1009600018B1FFF768FD00B1657100F033FC00F0CD
:100970009FFC80B1FFF767FC68B1022001F08CFAA0
:1009800094F90500401C03D10C488069FFF754FC22
:100990000120607004E0022001F07EFA657065714C
:1009A000FFF78FFD0000094068C0072000C0092044
:1009B000A08601000400FA05BCC00720384F0000E3
:1009C0002DE9F047FE4A00234FF40077156A4FF4F3
:1009D000FF79C5F30724DFF8ECA34FF4E05CDFF800
:1009E000E883FA4E25E0B84216D213280CD014281A
:1009F0000CD048450CD0A0F58072FF3A0AD03E28B2
:100A000013D81AF8002011E0EAB20FE022460DE0F8
:100A100055220BE0AA2209E0604506D208EB00024D
:100A2000A2F5805292F8002E00E00022F254401C01
:100A30005B1C8B42D7D3BDE8F08770B5E04D2C6BC3
:100A4000402C00D94024E86AE96902198A4202D997
:100A50000C1A042169702146FFF7B2FF2246DB49D8
:100A6000822001F0F2F8E86A2044E862286B011B5A
:100A7000D74829638268A2EB0402826005D06978B6
:100A8000022901D00021017370BD03216970F9E7CB
:100A9000CF4910B5CF4808600D22822001F0D5F86B
:100AA000C7490520487010BD70B50D46CA49496D4B
:100AB000490521D4B0F5007F1ED3C849C04CB0F51C
:100AC000E05F1AD28A68A369D21AC54B9A4204D34E
:100AD0008968A161002161606161BD4900235F39BE
:100AE000B94A07E0C4181444CE5CA4F580545B1CDA
:100AF00084F8006EAB42F5D370BD626922B98A6892
:100B0000A2618A686261A060B64A5279002AF3D174
:100B10008A686369D21AB44B9A421CD2B34B012241
:100B20001A708A68A26189686161A168401A616867
:100B3000884203D9616A884200D26060062001F0D1
:100B4000ABF961682A46BDE87040A14801F5005143
:100B50005F3800F05CBBBDE870400C2001F09CB930
:100B600010B5974CA178E06A4218E1698A4206D92B
:100B7000081AA07005206070022001F021F8A17809
:100B8000E06AFFF791FFA178E06A0844E062206B19
:100B9000421A8F4822638368A3EB0101816002D06F
:100BA0006178052904D100210173BDE810406FE789
:100BB00010BD2DE9F041824CA178E06A4218E1694C
:100BC0008A4206D9081AA07005206070022000F041
:100BD000F7FF7F4D0021A0787C4B5F3DE26A08E083
:100BE00056186F5C9E5DBE4202D00021A16202E0F9
:100BF000491C8142F4D31118E162216B0A1A74492D
:100C000022638B68A3EB0000886002D0607805281F
:100C100008D1A06A20B100200873BDE8F04137E791
:100C20000120F9E7BDE8F081694810B51F38D0F818
:100C30001110027D09BA21F0FF011143604A4902F7
:100C4000D162C18A49BA49021163806888420CD0D6
:100C5000822000F0B5FF022000F0B2FF5C490220C4
:100C60000873FFF715FF002010BD012010BD70B5FF
:100C70005748574D1F380224816829B1007B000670
:100C800007D4022000F09CFF2C73FFF701FF002027
:100C900070BD012070BD10B54D48494C1F388068AB
:100CA000A178884200D2A0704949A2785F39822099
:100CB00000F0CBFF032060704548A2788168891A54
:100CC00081600021017310BD414810B51F38816853
:100CD00039B1007B000601D5822000E0022000F03F
:100CE0006FFF3B4900200873BDE81040D0E610B507
:100CF000FFF7BDFF00281FD0354870215F38022262
:100D00000170002141708270C17001714171817167
:100D10000A22C271017241728172C1723022027361
:100D2000012242738173C1730174417424491220FA
:100D30008870BDE81040AEE710BD1CB5FFF797FF07
:100D400000286AD02A480A2206210388684600F053
:100D500025FA1F4800225F3880230270437082709A
:100D60000121C1702021017143718271C271412240
:100D70000272542242724F2282724C22C27201735A
:100D800041738173C17346220274502343747223EA
:100D900083746923C3746E2303757423437581754B
:100DA000C2756C22027661224276732282766822B4
:100DB000C276017741778177C1779DF8011019E0FC
:100DC00078C00720F84E000041C20720B9DC072098
:100DD000A0DC07205553425300C009200000094001
:100DE000A0860100BCC0072020A1070068C0072022
:100DF0000404000080F820109DF8021080F82110F3
:100E00009DF8031080F822109DF8041080F823103C
:100E1000DE4924208870FFF73EFF1CBD10B5FFF7A8
:100E200026FF00280CD0DA48032101700021417010
:100E30008170C170D54904208870BDE810402AE750
:100E400010BD10B5FFF713FF002810D0D0480021C7
:100E50000622017042708170C1700171417181710F
:100E6000C171CA4908208870BDE8104013E710BD61
:100E700010B5FFF7FCFE002815D0C44AC448116A1B
:100E8000491E0B0E03700B0C43700B0A8370C1706C
:100E900000210171417102238371C171082090709A
:100EA000BDE81040F7E610BD10B5FFF7E0FE0028E2
:100EB00019D0B7480021B54B0170417081700822EC
:100EC000C2701A6A140E0471140C4471140A8471ED
:100ED000C2710222027241728272C1720C20987039
:100EE000BDE81040D7E610BD2DE9F041A74DA84C54
:100EF0000021A8784034A64A02E0535C6354491CA0
:100F000003468142F9D31F2B72D12068A149884240
:100F10006ED19F4E60685F364FF001087060A06828
:100F2000B060607B18B9A07B08B1102802D986F8A0
:100F30000C8059E0E07B1E28F9D00FDC12282ED05F
:100F400005DC48B30328F2D1BDE8F041CFE615280F
:100F5000EDD01A28EBD1BDE8F0415FE702272A283F
:100F600028D010DC23281DD025281ED02828DED12B
:100F7000FFF75AFE002826D0207B000618D56F7098
:100F8000BDE8F04159E52F281ED05528CFD05A286A
:100F9000CDD1BDE8F04154E7BDE8F04194E6BDE8AD
:100FA000F041CAE6BDE8F0417EE7BDE8F0415FE709
:100FB000022016E0FFF738FE002804D0207B000650
:100FC0000ED485F801802DE6FFF72EFE0028FAD01A
:100FD000207B000604D485F80180C5F8288021E62E
:100FE000822000F0EDFD3773BDE8F04150E5FFE7EA
:100FF000822000F0E5FD022000F0E2FD062068708E
:1010000010E6624810B54178022908D003290ED0B5
:1010100004290FD0052901D10021417010BD5C4881
:101020004030C07B2828F9D1BDE8104005E5BDE877
:1010300010402DE5822000F0C3FDF8E710B55449BB
:10104000022000F0D1FD51498870487858B101283C
:101050000CD0022000F0B4FD4D4902205F3108732E
:10106000BDE8104014E5BDE810403DE74848403079
:10107000C07B2A2804D02F2805D1BDE8104098E570
:10108000BDE810406CE510BDFFB50246002002EB44
:10109000420501464FF440566C4603AA6B1844F8CB
:1010A0002130B34202DD002004B0F0BD3A4F07EB1F
:1010B0006307DB073F78575401D03B095354535C17
:1010C0008F0003F00F035354BB40491C18440329FD
:1010D000E4DBE9E7F0B506460020034602462E4C65
:1010E0004FF4007700E05B1CF55C45B102EB030CAC
:1010F000A4440CF5805C9CF800C8AC45F3D0032BED
:101100003FD302F5C0502044037F457FC67F03EBE9
:101110000523857F2D0405EB06652B4451EA030565
:101120002BD021B91949496840318B4225D8184B39
:1011300000216C335518254405F5805595F8005865
:101140005D54491C0C29F5D3817EC27E01EB02213E
:10115000027D407D120402EB00600C182046FFF770
:1011600093FF40F6F57501E0FFF78EFFC11EA9421F
:10117000FAD3A0F57061FF3901D00020F0BD204600
:10118000F0BD2032BA42AFD3F0BD000078C00720D6
:1011900041DC07205553424341C20720FFB5B2A6A8
:1011A0000446E1CE8DE8E100022902DA002004B015
:1011B000F0BD6018002100F8011D6946B3FBF2F58F
:1011C00002FB1535B3FBF2F34D5D00F8015DA04263
:1011D000F4D8ECE710B503F0C8FA03F0B2FAA64968
:1011E0004FF40052C1E90020A0F5F420886010BD42
:1011F00070B5034608468D189F49002449688D4202
:1012000000D9881A194603F0FFFA204670BDF8B5D8
:101210001446994E0A460B19716800258B4200D975
:101220000A1B03460094306803F019FB2846F8BDFA
:1012300010B50B4601460024184603F0B9FA2046C3
:1012400010BD2DE9FC410746002090460E46ADF842
:10125000000004460EE0351B402D00D94025391909
:101260002A468648FFF7E4FFAAB284496846FEF79B
:101270003BFF2C44B442EED33919424601A8FFF794
:10128000D7FFBDF80000BDF80410884202D101204C
:10129000BDE8FC810020FBE70021425C12B9491C3B
:1012A0001829FAD3182901D000207047012070476F
:1012B0002DE9F043704C00200C348BB0A070E0702E
:1012C000DFF8BC816F4F4FF4005620714FF48079E6
:1012D0000125192231466846FFF7AAFF022216218E
:1012E0003046FFF7AEFF00287ED0DDF80E10022258
:1012F00006F11900FFF7A5FF002875D09DF8001032
:1013000006292AD2DFE801F02A03032A2A1CD8F88A
:101310007420DDF80A30521C93421ED2D8F87400B3
:10132000DDF80A30C01ADDF80E30401C984214D3A4
:10133000DDF80A00DDF80E30184490420DD80DE0BB
:10134000DDF80E00B0F5F42F00D9A570DDF812001D
:10135000C0F30B40B0F5907F00D0A570012903D0F9
:10136000022901D0052943D19DF808004A464007CB
:1013700006F2194107D54448FFF75AFF4149424850
:10138000FEF7C5FE02E03F48FFF752FF002009903C
:10139000B888ADF824000999019889B2884200D034
:1013A000A57000200990387B8DF824000999BDF8BC
:1013B0000100C9B2884200D0A5709DF80000022843
:1013C00016D1386B0990DDF812000999884200D0D7
:1013D000A5700020099097F834008DF82400099931
:1013E0009DF80300C9B200E026E0884200D0A57055
:1013F0009DF81800401EFE2800D2A570BDF801001F
:10140000A0F57F41FF3901D04B2802D19DF80300A0
:1014100020B96846FFF740FF00B9A570DDF80E005F
:101420001B3606446846FFF737FF30B1E07880B1DD
:10143000217988420DD012E0A5709DF8180010B9EE
:101440002079401C2071E078401CC0B2E0700C286C
:1014500001D3A57003E0A07800283FF43AAFA0784C
:101460000BB0BDE8F083000030313233343536370D
:101470003839414243444546B0C00720B9DC072013
:10148000B04F0000B9DE0720B9DD0720FA4800217F
:101490004FF00112818001704170C0E90221704754
:1014A000F5491C31002000F09FBB10B5F24C1434FC
:1014B000A288402A00D940228020216800F0C5FB84
:1014C000216801442160A188081AA08010BD10B5D0
:1014D000E94C00201434216800F086FB21680144A7
:1014E0002160A188081AA08010BD0022114680202A
:1014F00000F0ABBBE149002000F076BB70B5DE48E0
:10150000DD4D1C3005F11405007810F01F040AD0E1
:10151000D949DA4B01F11C004A780079012C06D038
:10152000022C26D109E0D448001D28601DE002B33A
:10153000897888421DD2002015E000F08F04200633
:1015400005D504F00F064FF48030B04001E00120D3
:10155000A0400AB922070CD18A68024209D0C968A2
:101560000142E8D0012018802B60FFF79EFF012088
:1015700070BD002070BD024670B5BF48BE4C1C3027
:10158000017811F01F030146498804D0012B29D0AE
:10159000022B27D111E0012924D132B1012000F022
:1015A000BDFAA08840F0020005E0002000F0B6FA85
:1015B000A08820F00200A08021E0007900F08F00D8
:1015C000030605D500F00F034FF480359D4001E080
:1015D0000125854063782BB1030703D0A3682B4214
:1015E00000D009B1002070BD22B100F0E9FAE06836
:1015F000284303E000F0EEFAE068A843E060012031
:1016000070BD9D4810B51C30007810F01F0F9A482F
:1016100000F11C00C0782AD197491431012807D065
:1016200001F108020228937806D003281FD112E0A6
:1016300093480860122012E09248002204E00478E7
:101640000CB144882044521C9342F8D1027872B104
:101650000860408803E08C481844086000788A8855
:10166000824200D98880FFF720FF012010BD0020B2
:1016700010BD2DE9F84F804F00201C370090B8783E
:101680007D4E4FF000094FF0010A4FF4803B0028D7
:101690006BD07C4C65E06078022804D0042841D0EF
:1016A00005285CD141E06179B878814238D1707009
:1016B0002079B0707049002011F1100101F80090FC
:1016C000401C0428FAD301254FEA06080AFA05F05F
:1016D000D8F80810084202D0284600F05DFAD8F881
:1016E00008100BFA05F0084203D045F0800000F026
:1016F00053FA6D1C102DE9D34FF00110C8E902090F
:10170000012000F00CFAE0794006B8F8040002D598
:1017100040F0010001E020F00100A8F804001EE004
:1017200060881DE0E078009019E00098B8B9A078D2
:1017300000F08F05280604D505F00F010BFA01F023
:1017400001E00AFA05F0B16801432046B16000F0FB
:10175000FCF9284600F016FA284600F027FA20780F
:1017600004442078002896D11FE086F801900124D7
:101770005546D846B16805FA04F0084202D0204622
:1017800000F00AFAB16808FA04F0084203D044F005
:10179000800000F001FA641C102CEBD34FF0011014
:1017A000C6E90209002000F0BAF9B87871788842D9
:1017B00002D10120BDE8F88F0020FBE72DE9FC5F96
:1017C0002D4D00273E466878BB46B846002871D0AC
:1017D000BA462C4C05F11C0968E06078022804D058
:1017E000042808D005285FD119E06079697888421B
:1017F0005AD0608859E0A77899F80410E6784FF03D
:101800000008B94250D199F80200B0424CD11A48B0
:101810004FF0010A103010F807B0C65544E099F8AF
:101820000410B94240D1A17801F08F01019109065D
:1018300005D5019901F00F024FF4803101E0019AC2
:1018400001219140009199F80200B0421ED1A86890
:101850000843A860E968009881432046E96000F0E9
:1018600074F9019800F08EF9019800F09FF9009941
:1018700048EA010818E00000CCC00720E4E0072097
:10188000285000003A5000005B5000005E450BD12C
:1018900018EA010F08D1A8688843A860E86888435F
:1018A000E860019800F078F9207804442078002856
:1018B00093D15046BDE8FC9F2DE9F041494C0027EB
:1018C000A4F108062178A4F11C05082863D2DFE8FA
:1018D00000F06204647262628381FFF7E1FD2078A8
:1018E000C00900F04EF9E088B0802078C0F34111C3
:1018F000F1BB61780C294AD2DFE801F00609490BF7
:1019000049101A1D1F253142FFF7F8FD4DE0002058
:1019100000E00120FFF72FFE50B306E010F01F0F8C
:1019200035D1A07840F080002870BDE8F041DCE5BA
:10193000FFF767FE39E000202AE010F01F0F26D1E4
:1019400028481B381AE010F01F0F20D1FFF791FE36
:1019500070B1FFF7CAFDBDE8F041FEF70DBD00F024
:101960001F00012813D1687810B12079A97800E010
:101970000DE088420BD21B490C39084430601CE052
:1019800000F01F00012802D1FFF718FFC4E78020F4
:1019900000F016F9B780BDE8F081080608D4B088D9
:1019A0000028F8D0FFF793FDB0880028EFD0F2E7C9
:1019B000BDE8F0419EE5080602D5BDE8F04174E5BA
:1019C00028780106E7D500F07F002870BDE8F041D7
:1019D00000F054B8802000E00020BDE8F04100F0A5
:1019E000F9B80000E8C0072001460007C00E09064C
:1019F00000D5401C7047DA491022C1F80822C1F80E
:101A0000100200BFD1F80002C006FBD57047D44ACF
:101A10001023C2F80832C2F8100200BFD2F8000248
:101A2000C006FBD5C2F80832C2F81012D2F8000284
:101A3000C006FBD57047CA493022C1F80822C1F858
:101A4000100200BFD1F800028006FBD5D1F81402C5
:101A5000704710B5040001D0012000E000204FF4D1
:101A6000807141EA0041BF48FFF7D1FFBE494FF006
:101A700000700CB1886710BDC86710BD30B5BB4998
:101A8000BB4D41EA004421462846FFF7C0FF2146EE
:101A90002846BDE83040BAE7B1480021C0F84812F6
:101AA0004021C0F84C120122C0F84822C0F84C1264
:101AB000D0F80012C905FBD54FF0FF31C0F838123D
:101AC000C0F83412C0F808120C21C0F80412704794
:101AD000A84800B5C16821F0405141F00051C160F3
:101AE000C16C41F04051C164A3491A200860091D2E
:101AF0000A6830EA0202FBD14FF0E0214FF080701B
:101B0000C1F880029D4B202283F80024C1F8000117
:101B1000FFF7C2FF00205DF804EBAFE7704710B598
:101B200000B101204FF4807444EA00419448FFF76B
:101B30006EFF8B480321C0F8441200BFD0F800129A
:101B4000C905FBD5C0F8084210BD10B50246807823
:101B5000FFF74AFF8249D1F84432012484402343ED
:101B6000C1F84432C1F848029088C1F84C0200BF65
:101B7000D1F80002C005FBD54FF48070C1F808020F
:101B800010BD704700B5FFF72FFF7E495DF804EBED
:101B900041EA004089133AE700B5FFF725FF79498C
:101BA0005DF804EB41EA0040774930E700B5FFF704
:101BB0001BFF74495DF804EB41EA0040891326E7F6
:101BC00000B5FFF711FF6F495DF804EB41EA0040F3
:101BD0006E491CE700B5FFF707FF6A495DF804EBA3
:101BE00041EA0040891312E700F00F02012370B5AB
:101BF00003EB82035A4AC2F8283200BFD2F82032DF
:101C00001C05FBD5C3F309030024DD1C05E000BF60
:101C1000D2F8186241F8046B641CB4EB950FF7D34B
:101C20000021C2F8281241F24821C140C9070AD157
:101C3000FFF7DAFE4FF4A06141EA0040FFF7DBFE58
:101C40005348FFF7D8FE184670BD70B513460546D9
:101C5000434C00F00F00022202EB8000C4F828027F
:101C6000C4F824320020DA1C05E000BF51F8046BF0
:101C7000C4F81C62401CB0EB920FF7D30020C4F8EC
:101C800028022846FFF7B0FE4FF4A06141EA004069
:101C9000FFF7B1FE3F48FFF7AEFE184670BD2DE9D5
:101CA000F0412F4DD5F80032C5F80832180721D57C
:101CB0002C48FFF7A0FE3848FFF7BDFEC10605D54A
:101CC000FFF7EAFEBDE8F041FEF747BB810705D507
:101CD000BDE8F04100F00100FEF739BB010709D56E
:101CE000400703D5BDE8F041FEF73EBBBDE8F0413B
:101CF000FEF741BB294E58074FF001071CD4BDE841
:101D0000F0810024D5F8302207FA04F10A4210D0FD
:101D10006008C5F8381200BFD5F800128906FBD557
:101D2000D5F81412E2070CD056F8201009B10320A0
:101D30008847641C202CE5D3D5F830020028E0D178
:101D4000DDE73CB9490705D5316819B1012088475D
:101D50000124D7E756F820100029EAD00220E7E74F
:101D600000C000500005FE0000C0092000018000F6
:101D70000005D00000C00240F4CF005018E000E0A1
:101D80000005D8000005400000012000000101000E
:101D90000005F2000005FA000002FE00CC50000031
:101DA000002070479149820702D54FF48062CA63D0
:101DB000C20701D00222CA63420702D54FF4802233
:101DC000CA63020702D54FF40012CA63C20602D5E5
:101DD0004FF00072CA63800602D54FF08050C8638E
:101DE000002070478149820702D54FF480628A63E0
:101DF000C20701D002228A63420702D54FF4802233
:101E00008A63020702D54FF400128A63C20602D524
:101E10004FF000728A63800602D54FF080508863CD
:101E20000020704701460020704A8B0703D5536B92
:101E30005B0500D40220CB0704D0536B9B0701D471
:101E400040F001004B0704D5536B5B0301D440F015
:101E500004000B0704D5536B9B0201D440F008002B
:101E6000CB0604D5536B9B0101D440F010008906CA
:101E700004D5516BC90001D440F02000704710B563
:101E80000446FFF7CFFF0346FFF7ACFF24EA030049
:101E9000FFF788FF002010BD70B5554B50B1596851
:101EA000042403250226052907D2DFE801F00731C3
:101EB0005A819B0000205860986070BD042807D0AC
:101EC000052809D00124022808D001280BD015E0EC
:101ED0003F20FFF787FF56E001203AE03F20FFF761
:101EE00081FF022003E03F20FFF77CFF0120FFF786
:101EF00059FF3820FFF756FF5C6070BD0E28FCD1FB
:101F00003F20FFF76FFF0220FFF74CFF0120F1E7B2
:101F100006280AD0032810D00A2813D0092811D087
:101F20000D2819D00C28D3D070BD3F20FFF75AFFE1
:101F30000220FFF737FF5E6070BD3F20FFF752FFC2
:101F4000012031E03F20FFF74DFF0220FFF72AFF7D
:101F50003820BDE8704045E73F20FFF743FF0220EF
:101F600012E0062813D00A281AD00928BBD00C2862
:101F7000AED00D28F0D00F28DED13F20FFF732FF82
:101F80000220FFF70FFF0120BDE870400AE79868C4
:101F900010F01F0F00F101009860CDD102201EE06B
:101FA0003F20FFF71FFF0220FFF7FCFE5D6070BDC2
:101FB000072806D00A288BD00B288FD0092892D06A
:101FC00070BD0220FFF70EFF3820FFF70BFF986867
:101FD00010F03F0F00F101009860F1D10120BDE841
:101FE00070404CE70628A0D088E7000000C0092018
:101FF000F8C007204F4810B52021C0F8A01100BF3D
:10200000D0F8A0114906FBD50521C0F804114FF006
:102010004472C0F8A8214FF48062C0F8AC210122BC
:10202000C0F80C210B23C0F88430C0F88020AA220D
:10203000C0F88C205523C0F88C3000BFD0F8884001
:102040006401FBD50324C0F88040C0F88C20C0F8A0
:102050008C30C0F808113849C0F8C4104FF48271B0
:10206000C0F8C811D0F888106FEA11618A073349A7
:10207000D0F80C2102F0030207D07AB3012A44D031
:10208000022A47D0032A4ED13AE02AB1012A13D0BE
:10209000022A24D0032A46D1D0F88820D0F804316F
:1020A000C2F30742DBB2521C5B1C5A43D0F88830A3
:1020B000234CC3F30E030EE0D0F88820D0F804318F
:1020C000C2F30742DBB2521C5B1C5A43D0F8883083
:1020D0001C4CC3F30E035B1C634321E010E0D0F8FB
:1020E0008820D0F80431C2F30742DBB2521C5B1CDB
:1020F0005A43D0F888304FF47A44C3F30E03EAE72A
:10210000D0F80421104BD2B209E0D0F804210F4BD3
:10211000D2B204E0D0F804214FF4FA43D2B2521CF8
:10212000B3FBF2F20A60016821F4704141F40051FE
:10213000016010BD00C00F40DE96688704C1072013
:1021400000127A0000366E0100093D00001BB70046
:102150004FF0402100200867C86010224A61C86122
:10216000C022CA633F498A683F49C1E900203F490C
:1021700008603F49086078463E4908600020704783
:102180002DE9F04341F288320025384F384E394C62
:10219000904208D8642800D228B942F210729142C5
:1021A00001D8052907D2862038607846356020603E
:1021B0008620BDE8F083DFF8AC90D9F808302A4AD1
:1021C000D2F800C0A3EB0C03D2F804C00CEB4C080F
:1021D000C8EBCC1CB3EBCC0F06D205203860784698
:1021E000356020600520E4E74FF040234FF0020CFB
:1021F000C3F804C050B1DFF88080B8FBF0F04010A5
:102200009861D861C3F804C001205860D9F808006B
:10221000C2E900013D607846356020600020C8E7D3
:1022200070B5114C00250E466560FFF7A9FF0F49F8
:10223000000601D5086870BD0A4B06EB460220680F
:10224000C2EBC6129E68361AB6EBC20FFAD34FF035
:10225000402002224260C26B02F0FD02C263656050
:10226000E8E700000000094008C107206CC0072013
:1022700070C0072074C00720001BB700A8480021C9
:102280008162816821F040418160816C21F0404190
:1022900041F000418164A3494FF40042CA630A6AD5
:1022A00042F400420A62826822F440728260826CC8
:1022B00022F4407242F4007282641022CA630A6AF5
:1022C00042F010020A62026822F0300242F010026C
:1022D0000260026C22F0300242F0200202640268C6
:1022E00022F0C00242F040020260026C22F0C00202
:1022F0000264C26842F44032C260C26C22F44032CE
:1023000042F40032C264C26842F44042C260C26C0D
:1023100022F4404242F40042C264C26842F4407275
:10232000C260C26C22F4407242F40072C264C2689D
:1023300022F44052C260C26C22F44052C2644FF494
:1023400080028A630A6A42F480020A62C26822F446
:102350004012C260C26C22F44012C2644FF080622C
:102360008A630A6A42F080620A62426822F040622E
:1023700042F080624260426C22F0406242F00062B1
:102380004264426822F0405242F080524260426C05
:1023900022F0405242F000524264C26822F04052A1
:1023A00042F00052C260C26C42F04052C264C26944
:1023B00022F44022C261C26D42F44022C2654FF055
:1023C0000072CA670B6E43F000730B66036923F05B
:1023D00040730361036D43F0407303658314CB6561
:1023E0000B6C23F480530B64C36923F4401343F450
:1023F0000013C361C36D23F4401343F40013C3659A
:10240000036923F040630361036D23F040630365B8
:102410001313CB650B6C23F400530B64036923F493
:1024200040030361036D23F4400343F40003036599
:10243000C314CB650B6C23F400630B64836823F037
:1024400040538360836C23F0405343F00053836414
:10245000D312CB630B6A43F480430B62836823F48B
:1024600040138360836C23F4401343F400138364AC
:1024700003158B630B6A43F480630B62836823F05C
:102480000C038360836C23F00C0343F00803836424
:1024900002238B630B6A43F002030B62C36823F0D1
:1024A0003003C360C36C23F0300343F02003C364E4
:1024B000D3118B630B6A43F480230B62C36823F44C
:1024C0004063C360C36C23F4406343F40063C3649C
:1024D00013118B630B6A43F400130B62C36823F47C
:1024E0004023C360C36C23F4402343F40023C3643C
:1024F0008A630A6A42F000720A62C26822F040727D
:10250000C260C26C22F0407242F00072C2644FF0AE
:1025100080508863086A40F080500862704700006D
:1025200000C0024000C009201C484FF47A710068C6
:10253000B0FBF1F0B0F1807F0ED220F07F414FF080
:10254000E020491E4161164AF82182F8141D00213D
:102550008161072101617047FEE7124800B5022141
:1025600041600021016741610B22C260C16301210A
:102570004160FFF7D9FF002000BD0B480168491CEE
:10258000016000684FF4FA71B0FBF1F201FB120038
:10259000002802D10320FFF77FBC704704C1072049
:1025A0000FE000E00000094010C107201848022198
:1025B0000161072202600022426142624160C168FB
:1025C000C906FCD400E08168C1684907FBD400203B
:1025D00070470F498860C868C006FCD48868704797
:1025E00000B50B46024603E012F8010BFFF7F1FFBE
:1025F0005B1EF9D200BD00B50B46024604E0002088
:10260000FFF7E7FF02F8010B5B1EF8D200BD0000E8
:102610000080084070B500BF00BF00BF00BF00BF12
:1026200000BF00BF00BF00BF00BF00BF00BF00BFB2
:1026300000BF00BF00BF00BF00BF00BF00BF00BFA2
:1026400000BF00BF00BF00BF00BF00BF00BF00BF92
:1026500000BF00BF00BFFE4C4FF08065E563062061
:10266000FFF7B7FFA56300BF00BF00BF00BF00BFFB
:1026700000BF00BF00BF00BF00BF00BF00BF00BF62
:1026800000BF00BF00BF00BF00BF00BF00BF00BF52
:1026900000BF00BF00BF00BF00BF00BF00BF00BF42
:1026A00000BF00BF00BF70BD70B500BF00BF00BF5E
:1026B00000BF00BF00BF00BF00BF00BF00BF00BF22
:1026C00000BF00BF00BF00BF00BF00BF00BF00BF12
:1026D00000BF00BF00BF00BF00BF00BF00BF00BF02
:1026E00000BF00BF00BF00BF00BFD94C4FF08065E6
:1026F000E5630420FFF76DFFA56300BF00BF00BFC7
:1027000000BF00BF00BF00BF00BF00BF00BF00BFD1
:1027100000BF00BF00BF00BF00BF00BF00BF00BFC1
:1027200000BF00BF00BF00BF00BF00BF00BF00BFB1
:1027300000BF00BF00BF00BF00BF70BD70B5064640
:1027400000BF00BF00BF00BF00BF00BF00BF00BF91
:1027500000BF00BF00BF00BF00BF00BF00BF00BF81
:1027600000BF00BF00BF00BF00BF00BF00BF00BF71
:1027700000BF00BF00BF00BF00BF00BF00BF00BF61
:10278000B34D4FF08064EC635020FFF722FFAC6341
:1027900000BF00BF00BF00BF00BF00BF00BF00BF41
:1027A00000BF00BF00BF00BF00BF00BF00BF00BF31
:1027B00000BF00BF00BF00BF00BF00BF00BF00BF21
:1027C00000BF00BF00BF00BF00BF00BF00BF00BF11
:1027D00000BF00BF00BF00BF00BF00BF00BF00BF01
:1027E00000BF00BF00BF00BF00BF00BF00BF00BFF1
:1027F00000BF00BF00BF00BF00BF00BF00BF00BFE1
:1028000000BF00BF00BF00BF00BF00BF00BF00BFD0
:10281000EC630120FFF7DDFEB000FFF7DAFEAC63EA
:1028200000BF00BF00BF00BF00BF00BF00BF00BFB0
:1028300000BF00BF00BF00BF00BF00BF00BF00BFA0
:1028400000BF00BF00BF00BF00BF00BF00BF00BF90
:1028500000BF00BF00BF00BF00BF00BF00BF00BF80
:1028600070BD2DE9FE430F46044602A9794800F0E9
:10287000BCFD794D794EDFF8E88148B182202860AF
:102880002220794630608220C8F80010BDE8FE831F
:102890009DF80800800701D4FFF7BCFE02208DF8E8
:1028A0000000200C8DF80100200A8DF802008DF840
:1028B00003408DF8047000BF00BF00BF00BF00BF21
:1028C00000BF00BF00BF00BF00BF00BF00BF00BF10
:1028D00000BF00BF00BF00BF00BF00BF00BF00BF00
:1028E00000BF00BF00BF00BF00BF00BF00BF00BFF0
:1028F00000BF00BF00BF564F4FF08064FC6305214E
:102900006846FFF76DFEBC6300BF00BF00BF00BF9D
:1029100000BF00BF00BF00BF00BF00BF00BF00BFBF
:1029200000BF00BF00BF00BF00BF00BF00BF00BFAF
:1029300000BF00BF00BF00BF00BF00BF00BF00BF9F
:1029400000BF00BF00BF00BF002028607946306094
:10295000C8F800109AE72DE9FC5F3F4D3F4E404F0D
:102960005FEA020A8B4604464FF000080DD001A929
:10297000384800F03AFD80B1822028602120306084
:10298000784638608220BDE8FC9FC5F80080784614
:10299000C6F8008038600020F5E703208DF80000BD
:1029A000200C8DF80100200A8DF802008DF80340FC
:1029B00000BF00BF00BF00BF00BF00BF00BF00BF1F
:1029C00000BF00BF00BF00BF00BF00BF00BF00BF0F
:1029D00000BF00BF00BF00BF00BF00BF00BF00BFFF
:1029E00000BF00BF00BF00BF00BF00BF00BF00BFEF
:1029F000174C4FF08069C4F83C9004216846FFF7FB
:102A0000EFFD51465846FFF7F6FDC4F8389000BF79
:102A100000BF00BF00BF00BF00BF00BF00BF00BFBE
:102A200000BF00BF00BF00BF00BF00BF00BF00BFAE
:102A300000BF00BF00BF00BF00BF00BF00BF00BF9E
:102A400000BF00BF00BF00BF00BF00BF00BF9CE7CA
:102A500000C00920A08601006CC0072070C00720BC
:102A600074C007202DE9F05FFF4EDFF80094DFF817
:102A700000A4150083460F464FF000080ED0002436
:102A80000AE0395D0BEB0400FFF7EBFE000602D510
:102A90003068BDE8F09F641CAC42F2D3C6F80080F9
:102AA0007946C9F800800020CAF80010F1E72DE946
:102AB000FC47044601A9EF4800F097FCEA4DEB4EB5
:102AC000DFF8AC9348B1822028602220794630603C
:102AD0008220C9F80010BDE8FC879DF8040080073B
:102AE00001D4FFF797FD20208DF8000020098DF814
:102AF000010020018DF8020000248DF8034000BF82
:102B000000BF00BF00BF00BF00BF00BF00BF00BFCD
:102B100000BF00BF00BF00BF00BF00BF00BF00BFBD
:102B200000BF00BF00BF00BF00BF00BF00BF00BFAD
:102B300000BF00BF00BF00BF00BF00BF00BFDFF885
:102B400038834FF08067C8F83C7004216846FFF76F
:102B500047FDC8F8387000BF00BF00BF00BF00BF0E
:102B600000BF00BF00BF00BF00BF00BF00BF00BF6D
:102B700000BF00BF00BF00BF00BF00BF00BF00BF5D
:102B800000BF00BF00BF00BF00BF00BF00BF00BF4D
:102B900000BF00BF00BF2C60794634600020C9F838
:102BA000001098E72DE9FC478A46044601A9B14880
:102BB00000F01BFCAC4DAD4EDFF8B49240B182206A
:102BC00028602220794630608220C9F8001082E710
:102BD00003208DF8000020098DF8010020018DF8F8
:102BE000020000248DF8034000BF00BF00BF00BFFB
:102BF00000BF00BF00BF00BF00BF00BF00BF00BFDD
:102C000000BF00BF00BF00BF00BF00BF00BF00BFCC
:102C100000BF00BF00BF00BF00BF00BF00BF00BFBC
:102C200000BF00BF00BF00BFDFF84C824FF08067DD
:102C3000C8F83C7004216846FFF7D2FCB91350462F
:102C4000FFF7D9FCC8F8387000BF00BF00BF00BF55
:102C500000BF00BF00BF00BF00BF00BF00BF00BF7C
:102C600000BF00BF00BF00BF00BF00BF00BF00BF6C
:102C700000BF00BF00BF00BF00BF00BF00BF00BF5C
:102C800000BF00BF00BF00BF2C6079463460002049
:102C9000C9F800101FE72DE9F34F83B0044601A9DE
:102CA000744800F0A2FB704D704E714F4FF08208D7
:102CB00018B12120C5F800806CE09DF80400800761
:102CC00001D4FFF7A7FCAD208DF8000020098DF896
:102CD000010020018DF802004FF0000B8DF803B0C9
:102CE00000BF00BF00BF00BF00BF00BF00BF00BFEC
:102CF00000BF00BF00BF00BF00BF00BF00BF00BFDC
:102D000000BF00BF00BF00BF00BF00BF00BF00BFCB
:102D100000BF00BF00BF00BF00BF00BF00BF00BFBB
:102D2000DFF854914FF0806A5446C9F83CA0042162
:102D30006846FFF755FC02210498FFF751FCC9F8DB
:102D4000384000BF00BF00BF00BF00BF00BF00BFD2
:102D500000BF00BF00BF00BF00BF00BF00BF00BF7B
:102D600000BF00BF00BF00BF00BF00BF00BF00BF6B
:102D700000BF00BF00BF00BF00BF00BF00BF00BF5B
:102D800000BF022401A93B4800F02FFB48B12220DC
:102D9000C5F80080306078463860822005B0BDE814
:102DA000F08F00BF00BF00BF00BF00BF00BF00BF6B
:102DB00000BF00BF00BF00BF00BF00BF00BF00BF1B
:102DC00000BF00BF00BF00BF00BF00BF00BF00BF0B
:102DD00000BF00BF00BF00BF00BF00BF00BF00BFFB
:102DE00000BFC9F83CA0AD20FFF7F3FB0498022117
:102DF0002044FFF7F5FBC9F838A000BF00BF00BFB3
:102E000000BF00BF00BF00BF00BF00BF00BF00BFCA
:102E100000BF00BF00BF00BF00BF00BF00BF00BFBA
:102E200000BF00BF00BF00BF00BF00BF00BF00BFAA
:102E300000BF00BF00BF00BF00BFA41CA4B2B4F518
:102E4000805F9FD301A90B4800F0CFFA00287FF4E0
:102E500030AFFFF729FCC5F800B07846C6F800B0DF
:102E6000386000209AE700006CC0072070C007207F
:102E700074C00720A086010000C0092070B5FD4D78
:102E8000FD4EFE4C2AB1FFF766FD000609D520680D
:102E900070BD86202060092028607846306086203A
:102EA00070BD00202060286078463060002070BD32
:102EB0002DE9F04F89B0DFF8C483DFF8B8B35FEADB
:102EC00002094FF0000607910FD04FF480550146DC
:102ED0002A466846FDF704FADDE90047284601F076
:102EE00055FE5FEA000A0CD016E08621C8F80010F3
:102EF0000921CBF800107946DF480160862009B02F
:102F00004DE78221C8F800102221CBF80010794645
:102F1000D94801608220F2E7A9EB0605C7F5805089
:102F2000A84200D20546B5F5805F04D02046514640
:102F3000FFF738FE80B92046FFF7B9FD60B9079862
:102F40002A46811907EB0A00FDF72AFA2E4420468B
:102F50005146FFF7A0FE28B1504601F0EFFDD8F82A
:102F60000000CCE70027641C4E45D5D3504601F045
:102F7000E5FD0020C8F800007946CBF80000BE4807
:102F800001600020BBE72DE9FF4F8DB00D46DDF855
:102F900068900026B94C07935FEA09013FD04FF4CF
:102FA000805701463A466846FDF79AF9DDE900B1D7
:102FB0000C913A46691C6846FDF792F9DDE900106C
:102FC000CDE904013A4668460F99FDF789F9DDE934
:102FD000008500BFA9EB0607C5F58050B84200D2B6
:102FE000074625B1D8457CD10C98854279D14FF45C
:102FF000805001F0CBFD5FEA000A1BD0D8454FD1CD
:103000000C9885424CD12A464FEA08305146FFF7CA
:10301000A2FC000618D5504601F090FD79E086200C
:103020002060944809210160784693490860862011
:1030300011B0B4E6822020608E48222101607946DA
:103040008D4801608220F3E70598804509D10499F5
:1030500001EB0030C1F580525144FFF77CFC0006C3
:10306000D9D44046FFF723FD0006D4D407983A464A
:10307000811905EB0A00FDF793F9EA194FEA0830C8
:103080005146FFF7EFFC0006C5D40599884533D1BA
:10309000049800EB01300499C1F58052514427E0B7
:1030A000059988450AD1049800EB01300499C1F5CF
:1030B00080525146FFF74FFC0006ACD44046FFF764
:1030C000F6FC0006A7D407983A4681190F983044B9
:1030D000FFF7C8FC00069ED4059988450CD10498DA
:1030E00000E00DE000EB01300499C1F5805251463B
:1030F000FFF7B8FC00068ED4504601F01FFD0AE031
:1031000007983A4681190F983044FFF7ABFC000648
:1031100001D520688CE73E44002508F101084E45A2
:10312000FFF458AF534900202060086078465249A8
:10313000086000207CE72DE9F0474FF0000900BF50
:1031400000BF00BF00BF00BF00BF00BF00BF00BF87
:1031500000BF00BF00BF00BF00BF00BF00BF00BF77
:1031600000BF00BF00BF00BF00BF00BF00BF00BF67
:1031700000BF00BF00BF00BF00BF00BF00BF404E88
:103180004FF08065F5639F20FFF723FA0020FFF7DB
:1031900020FA00F0FF080020FFF71BFAC4B200205D
:1031A000FFF717FAC1B2B56300BF00BF00BF00BF91
:1031B00000BF00BF00BF00BF00BF00BF00BF00BF17
:1031C00000BF00BF00BF00BF00BF00BF00BF00BF07
:1031D00000BF00BF00BF00BF00BF00BF00BF00BFF7
:1031E00000BF00BF00BF00BF244D224E224FB8F1E8
:1031F000BF0F03D1252C0AD0262C08D082202860AE
:1032000021203060784638608220BDE8F0871D4874
:10321000412912D04FF48002422912D04A2910D0FD
:10322000C0F800900020FFF789FAC5F800907846B2
:10323000C6F8009038600020E7E74FF40011016005
:10324000F0E70260EEE72DE9F84F69460E4800F01E
:10325000CCF88227094C074D074E4FF0220A002870
:1032600062D19DF80000800701D4FFF7D3F900BFB9
:1032700000BF0BE070C0072074C007206CC007209F
:1032800000C0092014C10720A086010000BF00BFB4
:1032900000BF00BF00BF00BF00BF00BF00BF00BF36
:1032A00000BF00BF00BF00BF00BF00BF00BF00BF26
:1032B00000BF00BF00BF00BF00BF00BF00BF00BF16
:1032C00000BF00BF00BF00BFDFF8EC914FF0806887
:1032D000C9F83C806020FFF77CF9C9F8388000BF4E
:1032E00000BF00BF00BF00BF00BF00BF00BF00BFE6
:1032F00000BF00BF00BF00BF00BF00BF00BF00BFD6
:1033000000BF00BF00BF00BF00BF00BF00BF00BFC5
:1033100000BF00BF00BF00BF00BF00BF00BF6946C5
:10332000664800F062F838B127607846C5F800A01A
:1033300030608220BDE8F88F002020602860784649
:1033400030600020F6E75E48006870474FF4805018
:1033500070472DE9F04FDFF86C81DFF86CB189B070
:103360000F0004464FF0000626D04FF4805501466A
:103370002A466846FCF7B4FFDDE900A105912A461C
:10338000214606A8FCF7ACFFDDE906404FF0000936
:10339000BD1BC0F58051A94200D20D4620B1544555
:1033A00015D10599884212D12046FFF780FB00060F
:1033B0000DD5D8F80000A2E58621C8F80010092133
:1033C000CBF80010794641480160862097E52E44ED
:1033D000641C4846BE42DBD3C8F800007946CBF8EF
:1033E00000003A480160002089E52DE9F041384CA1
:1033F0000F460646A56806E0A068401BB04202D30F
:103400000120BDE8F081384600F003F80028F3D130
:10341000F7E770B5044600BF00BF00BF00BF00BFA4
:1034200000BF00BF00BF00BF00BF00BF00BF00BFA4
:1034300000BF00BF00BF00BF00BF00BF00BF00BF94
:1034400000BF00BF00BF00BF00BF00BF00BF00BF84
:1034500000BF00BF00BF184E4FF08065F563052028
:10346000FFF7B7F80020FFF7B4F82070B56300BF8E
:1034700000BF00BF00BF00BF00BF00BF00BF00BF54
:1034800000BF00BF00BF00BF00BF00BF00BF00BF44
:1034900000BF00BF00BF00BF00BF00BF00BF00BF34
:1034A00000BF00BF00BF00BF00BF00BF00BF20784B
:1034B00000F0010070BD000000C0092020A107003D
:1034C00014C107206CC0072070C0072074C00720FB
:1034D000000009402DE9FF4703A9FE4800F063FB07
:1034E000FD4DFE4EDFF8F89350B182202860212078
:1034F000794630608220C9F8001004B0BDE8F0873A
:103500009DF80C00800701D4FFF784F842208DF865
:1035100000000024CDF80140CDF80540ADF8094089
:1035200000BF00BF00BF00BF00BF00BF00BF00BFA3
:1035300000BF00BF00BF00BF00BF00BF00BF00BF93
:1035400000BF00BF00BF00BF00BF00BF00BF00BF83
:1035500000BF00BF00BF00BF00BF00BF00BF00BF73
:10356000DFF880834FF08067C8F83C700B21684615
:10357000FFF736F8C8F8387000BF00BF00BF00BFC3
:1035800000BF00BF00BF00BF00BF00BF00BF00BF43
:1035900000BF00BF00BF00BF00BF00BF00BF00BF33
:1035A00000BF00BF00BF00BF00BF00BF00BF00BF23
:1035B00000BF00BF00BF00BF2C6079463460002010
:1035C000C9F8001099E72DE9F34F85B0044603A927
:1035D000C04800F0E8FAC04DC04EC14F4FF0820B1A
:1035E00018B12120C5F800B060E0FFF713F84220C1
:1035F0008DF800004FF0000ACDF801A0CDF805A02D
:10360000ADF809A000BF00BF00BF00BF00BF00BFF2
:1036100000BF00BF00BF00BF00BF00BF00BF00BFB2
:1036200000BF00BF00BF00BF00BF00BF00BF00BFA2
:1036300000BF00BF00BF00BF00BF00BF00BF00BF92
:1036400000BF00BFDFF89C924FF08068C9F83C8053
:103650000B216846FEF7C4FFC9F8388000BF00BFE1
:1036600000BF00BF00BF00BF00BF00BF00BF00BF62
:1036700000BF00BF00BF00BF00BF00BF00BF00BF52
:1036800000BF00BF00BF00BF00BF00BF00BF00BF42
:1036900000BF00BF00BF00BF00BF00BF03A98D482F
:1036A00000F081FA48B12220C5F800B030607846B9
:1036B0003860822007B0BDE8F08F9DF80C008007CD
:1036C00001D4FEF7A7FF02208DF80000200C8DF832
:1036D0000100200A8DF8020006988DF803408DF84D
:1036E000040000BF00BF00BF00BF00BF00BF00BF9D
:1036F00000BF00BF00BF00BF00BF00BF00BF00BFD2
:1037000000BF00BF00BF00BF00BF00BF00BF00BFC1
:1037100000BF00BF00BF00BF00BF00BF00BF00BFB1
:1037200000BF4446C846C9F83C4005216846FEF73C
:1037300057FFC8F8384000BF00BF00BF00BF00BF40
:1037400000BF00BF00BF00BF00BF00BF00BF00BF81
:1037500000BF00BF00BF00BF00BF00BF00BF00BF71
:1037600000BF00BF00BF00BF00BF00BF00BF00BF61
:1037700000BF00BF00BFC5F800A07846C6F800A093
:103780003860002096E72DE9F05F534EDFF84C914A
:10379000DFF84CA1150083460F464FF000080ED00D
:1037A00000240AE0395D0BEB0400FFF70CFF000674
:1037B00002D53068BDE8F09F641CAC42F2D3C6F875
:1037C00000807946C9F800800020CAF80010F1E7AF
:1037D0002DE9F34F0024404D404E414FC3B0804689
:1037E0004FF0820A4FF0210BA14641A9394800F061
:1037F000DAF900287CD19DF80401800701D4FEF796
:1038000009FF02208DF800004FEA18108DF8010022
:1038100004EB08108DF8020044988DF8039000EB3B
:1038200004214FF4807201A8FCF7BAFD00BF00BF6D
:1038300000BF00BF00BF00BF00BF00BF00BF00BF90
:1038400000BF00BF00BF00BF00BF00BF00BF00BF80
:1038500000BF00BF00BF00BF00BF00BF00BF00BF70
:1038600000BF00BF00BF00BF00BF00BF1D494FF039
:103870008060C8634FF482716846FEF7B1FE194953
:103880004FF08060886300BF00BF00BF00BF00BF73
:1038900000BF00BF00BF00BF00BF00BF00BF00BF30
:1038A00000BF00BF00BF00BF00BF00BF00BF00BF20
:1038B00000BF00BF00BF00BF00BF00BF00BF00BF10
:1038C00000BF00BF00BF641CE4B2102C8DD341A91F
:1038D00000480AE0A08601006CC0072070C00720E5
:1038E00074C0072000C0092002E000F05CF940B17C
:1038F000C5F800A07846C6F800B03860822045B010
:10390000D9E6FEF7D1FEC5F800907846C6F80090DB
:1039100038600020F3E72DE9F04F89B0DFF85483D9
:10392000DFF854B35FEA02094FF0000607910FD0A9
:103930004FF4805501462A466846FCF7D1FCDDE984
:103940000047284601F022F95FEA000A0CD016E091
:103950008621C8F800100921CBF800107946C74825
:103960000160862009B0A6E68221C8F80010222155
:10397000CBF800107946C14801608220F2E7A9EB3C
:103980000605C7F58050A84200D20546B5F5805F10
:1039900004D020465146FFF705F980B92046FFF7CD
:1039A00086F860B907982A46811907EB0A00FCF7E8
:1039B000F7FC2E4420465146FFF70AFF28B1504637
:1039C00001F0BCF8D8F80000CCE70027641C4E4595
:1039D000D5D3504601F0B2F80020C8F8000079466F
:1039E000CBF80000A54801600020BBE72DE9FF4FA0
:1039F0008DB00D46DDF8689000269E4C07935FEA77
:103A000009013ED04FF4805701463A466846FCF71C
:103A100067FCDDE900B10C913A46691C6846FCF789
:103A20005FFCDDE90010CDE904013A4668460F99D4
:103A3000FCF756FCDDE90085A9EB0607C5F58050CB
:103A4000B84200D2074625B1D8457CD10C988542B2
:103A500079D14FF4805001F099F85FEA000A1BD049
:103A6000D8454FD10C9885424CD12A464FEA0830B0
:103A70005146FEF770FF000618D5504601F05EF87B
:103A800079E0862020607C480921016078467B49E6
:103A90000860862011B00EE6822020607648222140
:103AA00001607946754801608220F3E705988045FA
:103AB00009D1049901EB0030C1F580525144FEF761
:103AC0004AFF0006D9D44046FEF7F1FF0006D4D4E1
:103AD00007983A46811905EB0A00FCF761FCEA19E0
:103AE0004FEA08305146FFF74EFE0006C5D405994F
:103AF000884533D1049800EB01300499C1F5805218
:103B0000514427E0059988450AD1049800EB01301B
:103B10000499C1F580525146FEF71DFF0006ACD452
:103B20004046FEF7C4FF0006A7D407983A4681191D
:103B30000F983044FFF727FE00069ED4059988456C
:103B40000CD1049800E00DE000EB01300499C1F5C0
:103B500080525146FFF717FE00068ED4504600F003
:103B6000EDFF0AE007983A4681190F983044FFF7B5
:103B70000AFE000601D520688CE73E44002508F1C6
:103B800001084E45FFF458AF3B4900202060086013
:103B900078463A49086000207CE74FF4800070477F
:103BA0004FF4805070472DE9F041354C0F460646E2
:103BB000A56806E0A068401BB04202D30120BDE822
:103BC000F081384600F003F80028F3D1F7E770B52C
:103BD000044600BF00BF00BF00BF00BF00BF00BF62
:103BE00000BF00BF00BF00BF00BF00BF00BF00BFDD
:103BF00000BF00BF00BF00BF00BF00BF00BF00BFCD
:103C000000BF00BF00BF00BF00BF00BF00BF00BFBC
:103C100000BF1C4E4FF08065F5630520FEF7D9FC10
:103C20000020FEF7D6FC2070B56300BF00BF00BFC8
:103C300000BF00BF00BF00BF00BF00BF00BF00BF8C
:103C400000BF00BF00BF00BF00BF00BF00BF00BF7C
:103C500000BF00BF00BF00BF00BF00BF00BF00BF6C
:103C600000BF00BF00BF00BF00BF207800F0010010
:103C700070BD00006CC0072070C0072074C0072012
:103C80000000094000C009202DE9F047F74E8046AA
:103C90004FF080773068BC00F54DB84249D100BF85
:103CA00000BF00BF00BF00BF00BF00BF00BF00BF1C
:103CB00000BF00BF00BF00BF00BF00BF00BF00BF0C
:103CC00000BF00BF00BF00BF00BF00BF00BF00BFFC
:103CD00000BF00BF00BF00BF00BF00BF00BFEC635C
:103CE0001520FEF776FC0020FEF773FC00F0FF09BC
:103CF000AC6300BF00BF00BF00BF00BF00BF00BF7C
:103D000000BF00BF00BF00BF00BF00BF00BF00BFBB
:103D100000BF00BF00BF00BF00BF00BF00BF00BFAB
:103D200000BF00BF00BF00BF00BF00BF00BF00BF9B
:103D300000BF00BF00BF00BF00BF00BF00BF00BF8B
:103D400000BF00BF00BF00BF00BF00BF00BF00BF7B
:103D500000BF00BF00BF00BF00BF00BF00BF00BF6B
:103D600000BF00BF00BF00BF00BF00BF00BF00BF5B
:103D700000BFEC630620FEF72CFCAC6300BF00BF65
:103D800000BF00BF00BF00BF00BF00BF00BF00BF3B
:103D900000BF00BF00BF00BF00BF00BF00BF00BF2B
:103DA00000BF00BF00BF00BF00BF00BF00BF00BF1B
:103DB00000BF00BF00BF00BF00BF00BF00BF00BF0B
:103DC00000BF00BF00BF00BF00BF00BF00BF00BFFB
:103DD00000BF00BF00BF00BF00BF00BF00BF00BFEB
:103DE00000BF00BF00BF00BF00BF00BF00BF00BFDB
:103DF00000BF00BF00BF00BF00BF00BFEC630120D9
:103E0000FEF7E7FB4FEA8800FEF7E3FB3068B842B5
:103E100002D14846FEF7DDFBAC6300BF00BF00BF28
:103E200000BF00BF00BF00BF00BF00BF00BF00BF9A
:103E300000BF00BF00BF00BF00BF00BF00BF00BF8A
:103E400000BF00BF00BF00BF00BF00BF00BF00BF7A
:103E500000BF00BF00BF00BF00BFBDE8F0872DE975
:103E6000FC5F8846044601A9824800F05DFB824D54
:103E7000824E834FF0BB03208DF8000020098DF89F
:103E8000010020018DF802004FF000098DF8039029
:103E900000BF00BF00BF00BF00BF00BF00BF00BF2A
:103EA00000BF00BF00BF00BF00BF00BF00BF00BF1A
:103EB00000BF00BF00BF00BF00BF00BF00BF00BF0A
:103EC00000BF00BF00BF00BF00BF00BF00BF00BFFA
:103ED000DFF89CB14FF0806ACBF83CA00421684623
:103EE000FEF77EFB00240020FEF773FBC0B28DF8C6
:103EF000040000E003E018F80410884208D0822093
:103F0000286022203060784638608220BDE8FC9F1F
:103F1000641CB4F5805FE6D3CBF838A000BF00BFC7
:103F200000BF00BF00BF00BF00BF00BF00BF00BF99
:103F300000BF00BF00BF00BF00BF00BF00BF00BF89
:103F400000BF00BF00BF00BF00BF00BF00BF00BF79
:103F500000BF00BF00BF00BF00BF00BFC5F800909A
:103F60007846C6F8009038600020CFE72DE9F0478A
:103F70004FF0000900BF00BF00BF00BF00BF00BF7F
:103F800000BF00BF00BF00BF00BF00BF00BF00BF39
:103F900000BF00BF00BF00BF00BF00BF00BF00BF29
:103FA00000BF00BF00BF00BF00BF00BF00BF00BF19
:103FB00000BF00BF2E4E4FF08065F5639F20FEF7D7
:103FC00008FB0020FEF705FB00F0FF080020FEF7CD
:103FD00000FBC4B20020FEF7FCFAC1B2B56300BF1B
:103FE00000BF00BF00BF00BF00BF00BF00BF00BFD9
:103FF00000BF00BF00BF00BF00BF00BF00BF00BFC9
:1040000000BF00BF00BF00BF00BF00BF00BF00BFB8
:1040100000BF00BF00BF00BF00BF00BF00BF164D04
:10402000164E174FB8F1C20F01D1202C07D08220B5
:104030002860212030607846386082200DE70B48E8
:1040400014291FD0152920D0162922D0182923D0B1
:10405000C0F800900020FFF717FEC5F800907846E2
:10406000C6F8009038600020F7E6000018C107206D
:1040700000C00920A08601006CC0072070C0072086
:1040800074C007204FF4801101E04FF4001101606B
:10409000E0E74FF48001FAE74FF08071F7E72DE990
:1040A000F34FC3B0804600244FF0820AFE4DFF4E0E
:1040B000FF4F4FF0210BA14641A9FE4800F034FA12
:1040C00000286CD1FEF7A6FA02208DF800004FEA16
:1040D00018108DF8010004EB08108DF802004498C8
:1040E0008DF8039000EB04214FF4807201A8FCF7D7
:1040F00057F900BF00BF00BF00BF00BF00BF00BF37
:1041000000BF00BF00BF00BF00BF00BF00BF00BFB7
:1041100000BF00BF00BF00BF00BF00BF00BF00BFA7
:1041200000BF00BF00BF00BF00BF00BF00BF00BF97
:1041300000BFE1494FF08060C8634FF48271684668
:10414000FEF74EFADC494FF08060886300BF00BF85
:1041500000BF00BF00BF00BF00BF00BF00BF00BF67
:1041600000BF00BF00BF00BF00BF00BF00BF00BF57
:1041700000BF00BF00BF00BF00BF00BF00BF00BF47
:1041800000BF00BF00BF00BF00BF00BF641CE4B29F
:10419000102C91D341A9C74800F0C6F948B1C5F821
:1041A00000A07846C6F800B03860822045B0BDE86F
:1041B000F08FFEF779FAC5F800907846C6F80090BF
:1041C00038600020F2E72DE9F04F89B0DFF8D8829F
:1041D0005FEA020B4FF0000607910FD04FF48055B5
:1041E00001462A466846FCF77BF8DDE90047284689
:1041F00000F0CCFC5FEA00090CD016E08621AB4849
:10420000C8F80010092101607946A948016086209C
:1042100009B0CCE78221A548C8F80010222101602E
:104220007946A34801608220F2E7ABEB0605C7F5AB
:1042300080504FF0000AA84200D20546B5F5805FD5
:1042400004D020464946FEF7ADFCD8B907982A4667
:10425000811907EB0900FCF7A3F82046FEF727FCBD
:1042600080B920464946FFF71AFF58B9204649460B
:10427000FFF7F5FD78B10AF1010000F0FF0ABAF18D
:10428000030F05D3484600F059FCD8F80000BFE7FB
:10429000BAF1000FE1D12E440027641C5E45C4D35F
:1042A000484600F04BFC81490020C8F80000086037
:1042B00079467F4801600020AAE72DE9FF4F8DB0C5
:1042C0000D46DDF868900026774C07935FEA0901F8
:1042D0003FD04FF4805701463A466846FCF700F855
:1042E000DDE900B10C913A46691C6846FBF7F8FF1E
:1042F000DDE90010CDE904013A4668460F99FBF765
:10430000EFFFDDE9008500BFA9EB0607C5F580508A
:10431000B84200D2074625B1D8457CD10C988542D9
:1043200079D14FF4805000F031FC5FEA000A1BD0D5
:10433000D8454FD10C9885424CD12A464FEA0830D7
:104340005146FEF708FB000618D5504600F0F6FB74
:1043500079E086202060554809210160784654495B
:104360000860862011B022E7822020604F48222179
:10437000016079464E4801608220F3E70598804548
:1043800009D1049901EB0030C1F580525144FEF788
:10439000E2FA0006D9D44046FEF789FB0006D4D4E1
:1043A00007983A46811905EB0A00FBF7F9FFEA196D
:1043B0004FEA08305146FFF7E6F90006C5D40599E3
:1043C000884533D1049800EB01300499C1F580523F
:1043D000514427E0059988450AD1049800EB013043
:1043E0000499C1F580525146FEF7B5FA0006ACD4E7
:1043F0004046FEF75CFB0006A7D407983A468119B1
:104400000F983044FFF7BFF900069ED40599884500
:104410000CD1049800E00DE000EB01300499C1F5E7
:1044200080525146FFF7AFF900068ED4504600F097
:1044300085FB0AE007983A4681190F983044FFF748
:10444000A2F9000601D520688CE73E44002508F15A
:1044500001084E45FFF458AF144900202060086061
:1044600078461349086000207CE7144800687047CC
:104470004FF4805070472DE9F04FDFF82C80DFF8C3
:104480002CB089B00F0004464FF0000633D04FF433
:10449000805501462A466846FBF722FFDDE900A168
:1044A00005912A4621460BE06CC0072070C007200A
:1044B00074C00720A086010000C0092018C1072091
:1044C00006A8FBF70DFFDDE906404FF00009BD1B14
:1044D000C0F58051A94200D20D4620B1544515D1F6
:1044E0000599884212D12046FEF7E1FA00060DD563
:1044F000D8F800008CE68621C8F800100921CBF816
:10450000001079463B480160862081E62E44641CF9
:104510004846BE42DBD3C8F800007946CBF800001D
:1045200034480160002073E62DE9F041324C0F461B
:104530000646A56806E0A068401BB04202D30120F1
:10454000BDE8F081384600F003F80028F3D1F7E722
:1045500070B5044600BF00BF00BF00BF00BF00BF72
:1045600000BF00BF00BF00BF00BF00BF00BF00BF53
:1045700000BF00BF00BF00BF00BF00BF00BF00BF43
:1045800000BF00BF00BF00BF00BF00BF00BF00BF33
:1045900000BF00BF194E4FF08065F5630520FEF7A0
:1045A00018F80020FEF715F82070B56300BF00BFB3
:1045B00000BF00BF00BF00BF00BF00BF00BF00BF03
:1045C00000BF00BF00BF00BF00BF00BF00BF00BFF3
:1045D00000BF00BF00BF00BF00BF00BF00BF00BFE3
:1045E00000BF00BF00BF00BF00BF00BF207800F0C9
:1045F000010070BD74C007200000094000C0092000
:1046000000207047AE4982200860AE492120086032
:104610007846AD49086082207047A9498220086029
:10462000A849222008607846A74908608220704780
:10463000A34982200860A349222008607846A24945
:1046400008608220704770B5002400BF00BF00BF23
:1046500000BF00BF00BF00BF00BF00BF00BF00BF62
:1046600000BF00BF00BF00BF00BF00BF00BF00BF52
:1046700000BF00BF00BF00BF00BF00BF00BF00BF42
:1046800000BF00BF00BF00BF00BF904E4FF080656D
:10469000F5639F20FDF79DFF0020FDF79AFF60F373
:1046A00007040020FDF795FF60F30F240020FDF7BD
:1046B00090FF60F31744B56300BF00BF00BF00BFA9
:1046C00000BF00BF00BF00BF00BF00BF00BF00BFF2
:1046D00000BF00BF00BF00BF00BF00BF00BF00BFE2
:1046E00000BF00BF00BF00BF00BF00BF00BF00BFD2
:1046F00000BF00BF00BF00BF7549601A8C421AD0CE
:104700000BDCA4F1C204B4F5A11414D0B4F5803FBD
:1047100011D0B4F5003F0BD10DE06E49401805D023
:104720006D49401809D06D49C84201D1022400E00A
:104730000024204670BD0324FBE70424FEF7CAFED4
:10474000F7E76748007828B1664900EBC00051F8E8
:10475000200000475A49822008605A4921200860F9
:104760007846594908608220704770B5FFF76BFFA3
:104770005B49544D544E524C087050B1594900EBAE
:10478000C00001EB800080688047000609D52068E2
:1047900070BD822020602120286078463060822011
:1047A00070BD00202060286078463060002070BD19
:1047B0002DE9F0414A4B434D434E1B78404C63B1C9
:1047C0009AB1484F03EBC30307EB83031B69984778
:1047D000000612D52068BDE8F081822020602120EB
:1047E0002860784630608220F5E786202060092026
:1047F0002860784630608620EDE700202060286041
:10480000784630600020E6E72DE9F041344B2D4D2D
:104810002D4E1B782A4C5BB192B1324F03EBC30390
:1048200007EB83039B699847000611D52068D2E700
:104830008220206022202860784630608220CAE7EB
:104840008620206009202860784630608620C2E7F4
:10485000002020602860784630600020BBE7F8B573
:104860001F4C184D184E2778154CDDF818C087B12D
:10487000BCF1000F15D0CDF800C0DFF868C007EB21
:10488000C7070CEB8707FF69B847000611D52068FA
:10489000F8BD822020602220286078463060822087
:1048A000F8BD862020600920286078463060862088
:1048B000F8BD002020602860784630600020F8BDF8
:1048C0006CC0072070C0072074C0072000C00920FA
:1048D000C220180003FBD6FF00FFFEFF0001F8FF17
:1048E0001CC107200C51000070B50024254600288B
:1048F00001DA01244042002901DA01254942FBF78F
:1049000061FDAC4200D04042002C00D0494270BD55
:10491000064C074D06E0E06840F0010394E807000C
:1049200098471034AC42F6D3FBF7D4FBE4510000B7
:10493000145200000FB41CB50A46521ECDE9000205
:1049400007A9054B6A46069800F010F8009A002166
:1049500011701CBC5DF814FB254B0000002001E029
:1049600001C1121F002AFBD1704700002DE9FF4F43
:104970008BB09A460F460546002606E025280BD048
:1049800052460D9990476D1C761C28780028F5D169
:104990000FB03046BDE8F08F0024A04601226049E8
:1049A00000E0044315F8013F203B02FA03F00842FF
:1049B000F7D128782E2817D115F8010F44F00404F8
:1049C0002A280ED06FF02F022878A0F13001092993
:1049D0000AD808EB880102EB410100EB01086D1CCD
:1049E000F2E757F8048B6D1C287869283ED006DC66
:1049F0000028CDD063280BD0642804D136E073287A
:104A000010D075284BD052460D999047761C85E002
:104A100017F8040B8DF8000000208DF80100E9461E
:104A2000012003E057F8049B4FF0FF3061074FF07F
:104A3000000401D40AE0641C44450DDA8442FADB28
:104A400019F804100029F6D106E0641C8442FCDB4E
:104A500019F804100029F8D1264404E019F8010BD4
:104A600052460D999047641EF8D257E001CF4FF09F
:104A70000A0B002802DA40422D2102E0210504D56C
:104A80002B218DF82410012103E0E10705D020211E
:104A9000F7E70DF1200908910CE00021F9E701CFBB
:104AA0004FF00A0BF9E75946FBF78CFC01F1300295
:104AB00009F8012D0028F6D1ADEB090000F1200B1B
:104AC000600701D44FF00108D84502DDA8EB0B00C8
:104AD00000E000208046002406E009A85246005D60
:104AE0000D999047641C761C08988442F5DB04E01D
:104AF000302052460D999047761CB8F10001A8F17C
:104B00000108F5DC05E019F8010B52460D999047B4
:104B1000761CBBF10001ABF1010BF4DC6D1C34E73A
:104B2000092801004A68002A06D00A68531C0B6055
:104B300010704868401E48607047000010B500289B
:104B400021D0114B0022001F196803E0814203D8D5
:104B50000A4649680029F9D152B11368841A9C4267
:104B600004D1006818441060104602E0506000E074
:104B7000186039B102680B1A934203D10B681A44CA
:104B800002604968416010BD20C10720F0B50B30BC
:104B9000154D20F007010024144A0FE003688B42F2
:104BA0000BD38B4205D95E1A43184768C3E90067E7
:104BB00000E04368136002C004E0021D1068002892
:104BC000ECD12046002802D1286808B10020F0BDB1
:104BD000064A07481060074A121A22F00702C0E985
:104BE000002401202860D7E724C1072020C1072026
:104BF000040000100050001000050F0A1B1E1411C5
:104C000033363C39282D272263666C69787D7772AC
:104C100050555F5A4B4E4441C3C6CCC9D8DDD7D29C
:104C2000F0F5FFFAEBEEE4E1A0A5AFAABBBEB4B18C
:104C300093969C99888D878283868C89989D97927C
:104C4000B0B5BFBAABAEA4A1E0E5EFEAFBFEF4F16C
:104C5000D3D6DCD9C8CDC7C240454F4A5B5E54515C
:104C600073767C79686D676223262C29383D37324C
:104C700010151F1A0B0E040103060C09181D17123C
:104C800030353F3A2B2E242160656F6A7B7E74712C
:104C900053565C59484D4742C0C5CFCADBDED4D11C
:104CA000F3F6FCF9E8EDE7E2A3A6ACA9B8BDB7B20C
:104CB00090959F9A8B8E848180858F8A9B9E9491FC
:104CC000B3B6BCB9A8ADA7A2E3E6ECE9F8FDF7F2EC
:104CD000D0D5DFDACBCEC4C143464C49585D5752DC
:104CE00070757F7A6B6E646120252F2A3B3E3431CC
:104CF00013161C19080D0702000021104220633012
:104D00008440A550C660E770088129914AA16BB123
:104D10008CC1ADD1CEE1EFF13112100273325222CB
:104D2000B5529442F772D662399318837BB35AA373
:104D3000BDD39CC3FFF3DEE362244334200401149B
:104D4000E664C774A44485546AA54BB528850995C3
:104D5000EEE5CFF5ACC58DD553367226111630066B
:104D6000D776F6669556B4465BB77AA71997388713
:104D7000DFF7FEE79DD7BCC7C448E5588668A7782B
:104D80004008611802282338CCC9EDD98EE9AFF963
:104D9000488969990AA92BB9F55AD44AB77A966A0B
:104DA000711A500A333A122AFDDBDCCBBFFB9EEBB3
:104DB000799B588B3BBB1AABA66C877CE44CC55CDB
:104DC000222C033C600C411CAEED8FFDECCDCDDD03
:104DD0002AAD0BBD688D499D977EB66ED55EF44EAB
:104DE000133E322E511E700E9FFFBEEFDDDFFCCF53
:104DF0001BBF3AAF599F788F8891A981CAB1EBA1A7
:104E00000CD12DC14EF16FE18010A100C230E32022
:104E10000450254046706760B9839893FBA3DAB3CA
:104E20003DC31CD37FE35EF3B1029012F322D23272
:104E30003542145277625672EAB5CBA5A89589859A
:104E40006EF54FE52CD50DC5E234C324A0148104C2
:104E50006674476424540544DBA7FAB79987B8976A
:104E60005FE77EF71DC73CD7D326F2369106B01612
:104E700057667676154634564CD96DC90EF92FE92A
:104E8000C899E9898AB9ABA9445865480678276862
:104E9000C018E1088238A3287DCB5CDB3FEB1EFB0A
:104EA000F98BD89BBBAB9ABB754A545A376A167AB2
:104EB000F10AD01AB32A923A2EFD0FED6CDD4DCDDA
:104EC000AABD8BADE89DC98D267C076C645C454C02
:104ED000A23C832CE01CC10C1FEF3EFF5DCF7CDFAA
:104EE0009BAFBABFD98FF89F176E367E554E745E52
:104EF000932EB23ED10EF01EEB3C904D53444F53D7
:104F0000352E3000020201000110000004F80C00F0
:104F1000010001000000000000000000000029EF77
:104F2000BEADDE41544F4C20465072696E7446410E
:104F3000543132202020000000000000001000004A
:104F40000020000000300000004000000050000081
:104F50000060000000700000008000000090000071
:104F600000A0000000B0000000C0000000D0000061
:104F700000E0000000F000000000010000800100DF
:104F80000000020000800200000003000080030017
:104F900000000400008004000000050000800500FF
:104FA00000000600008006000000070000800700E7
:104FB000FF0F0000FF1F0000FF2F0000FF3F000059
:104FC000FF4F0000FF5F0000FF6F0000FF7F000049
:104FD000FF8F0000FF9F0000FFAF0000FFBF000039
:104FE000FFCF0000FFDF0000FFEF0000FFFF000029
:104FF000FF7F0100FFFF0100FF7F0200FFFF0200B3
:10500000FF7F0300FFFF0300FF7F0400FFFF04009A
:10501000FF7F0500FFFF0500FF7F0600FFFF060082
:10502000FF7F0700FFFF0700120110010000004092
:1050300051C20313000104204801090220000101AC
:10504000008032090400000208065062070582024F
:105050004000000705020240000000040309041C90
:1050600003410054004F004C00200020002000208D
:1050700000200020002000200020002803460050CF
:1050800000720069006E007400200046006C006130
:105090000073006800200020002000200020002075
:1050A0000020001A034600690072006D007700615D
:1050B000007200650030003000300030000E034DFB
:1050C0000065006D006F007200790000B9180000E3
:1050D000000000007B030000000000000000000052
:1050E00000000000000000000000000000000000C0
:1050F00000000000000000000000000000000000B0
:105100000000000000000000000000000146000058
:1051100001460000054600001B4600000546000051
:105120001B4600001B4600001B46000031460000E5
:105130000146000001460000054600001B46000035
:10514000054600001B4600001B4600001B460000F1
:1051500031460000473300004D3300003731000076
:10516000473200007D2E0000B12E0000652A0000AD
:10517000872F0000533300006B440000714400008F
:105180006D3F0000473200007D2E0000C741000047
:1051900087370000BB420000774400009B3B0000C3
:1051A000A13B000037310000473200007D2E000097
:1051B0001739000087370000ED3900005333000035
:1051C00000000000000000000000000000000000DF
:1051D00000000000000000000000000000000000CF
:1051E000000000001452000000C007202801000049
:1051F000F0030000145200000000001000500000F6
:105200005C4900003C53000028C10720003000002A
:105210005C49000041544F4C20465072696E74281E
:1052200000000000000000000000D4284B3D0000FA
:10523000000000000000000000000000000000006E
:10524000000000000000000000000000000000005E
:10525000000000000000000000000000000000004E
:10526000000000000000000000000000000000003E
:105270000000000000C00720000000000000000047
:10528000000000000000000000000000000000001E
:10529000000000000000000000000000000000000E
:1052A00000000000000000000000000000000000FE
:1052B00000000000000000000000000000000000EE
:1052C00000000000000000000000000000000000DE
:1052D00000000000000000000000000000000000CE
:1052E00000000000000000000000000000000000BE
:1052F00000000000000000000000000000000000AE
:10530000000000000000000000000000000000009D
:10531000000000000000000000093D000000000047
:10532000000000000000000000000000000000007D
:10533000000000000000000000000000EB171765EF
:1053400080F64DC21FFD75889D4E7EA24184B9A393
:105350007208030D5B78A3E1C68ED9FDCD906D6018
:105360000AE0AEB82E950CC4A1C66F32BE54DDA5BE
:105370003E86FCC073DD5A6147B0D3F94BF8F16942
:10538000A1D10FE8C8D6B049AA92D63F2ACA753132
:10539000281227EB9EC376387F53E4EDBA1E55B52D
:1053A000A1A8B06F7CAFE560C253496FEE6BCD3101
:1053B000E3B656F9F13FFDE955E051757A0F4288A1
:1053C000BDDCE0B858AFFC63043B4BD8C7B856FA15
:1053D000C3AD3A35A2956CEBF0AE934F796CE49F78
:1053E0004D219B34E657C7EC9FE749C19E8816A420
:1053F00075C72698C77B9A5F94B353F618292FA1D7
:10540000D17FEB6584AE1C78F5E75BB18C4D210252
:105410007D0B7D7E7F1BF8F7721AE759DEB93C3CA5
:105420001A2813A23856E61D4D74DE060131774A5C
:10543000263FF0AF2BE30675B1118E03EC721A1EF6
:105440004586D26B9B2C1607394D1729526FD475A0
:105450006BE4478A2A571CC530B04DA41B585A67C5
:10546000A73D09C24D340516C02CA404B9C2BD5BCA
:105470002EA004B41755B955464E6E83CF8500371C
:105480008454153A6738C4D8B46EB5F88A3E5C11B6
:105490003BE97DBF232EB252A0C3C77C2C64E8AD8C
:1054A000C4F097630013667D4428F7F8DB989FA447
:1054B000AAFF4C3A603D1BD27856F499C9C3B0DFBD
:1054C000E4DAB73FA52DFDCD3154BAF84BA226EB57
:1054D00038B4FDDC8AA2A4DF2E63F0172AF86D38F9
:1054E000FF23AE6EBE98A45F869C5CD961DE3D5CF6
:1054F0000D63B2C41AF5CB97BA0BDA83DE108401C0
:105500002028ACAF203934EE92DAD236B99B29305C
:10551000CF82723ACB7C3C47C299A07F10A5068C03
:10552000A4AC236596C0E19ECEDA4AED6DDB721223
:1055300025500697B2598DCB62FBE649C2AE96481C
:10554000B58285EDA020A72F0F2ACC23BB15287884
:10555000E30A3A4A5AB43B3F92799D26C49A013FE6
:1055600032D9F9986D50587CFF7A4606D592441787
:105570004C0BEF7F2A7C6F6D7B3305759022ABE17E
:105580005703668B2CE96EE7AF185FA07373E129B0
:10559000B962A99F33EE34A9F04989BDEEC3552EF7
:1055A000EF252D5E1B072F4E03313DEA3292454A0F
:1055B0001FB8C5BD0669307A56468BE696BFBE2F2A
:1055C0004EAF5334B3613A036614A821D59AA53A75
:1055D0000733A1BFAA66F616D02093515221A4B07A
:1055E000A71E06E3D8169DDDBDC9AAA2FD00FE7761
:1055F000237E7FA483958CC682D2502059988385C0
:1056000059432486402BB1DBEFCC0F23325647FFA2
:105610009DAF04052AADF7FAA43C0B3E254565A2D3
:1056200077E82D0D73726374A4A05F906E7F0650AF
:1056300013212BA1ABCF98C3D45F44715D3BF1F331
:1056400080EC2D43B865815B4421954EA363440EE5
:105650009107DDE353D3D0BA821B3922B8C16A4225
:10566000E21D0D3015D7F017F86409B52083CD97EA
:105670009CE19B1B56CD143BC34B1F7D4C08BB9636
:105680002C581F327CCC7E664617D8FF382E5452D9
:1056900026FF4857E7B3B8B12A7A19B3F1F04EE9BB
:1056A00035981D10D479C4A3F1C3061E9D62B99329
:1056B000E33CE40AF6E7A34444931E1F4D00E7923F
:1056C000C1E06E172F752785C115BD63F4D41FD4B3
:1056D000E98D29FE87233410B03BE39D0E00656EF3
:1056E0009DA9DF1150A92F96125310B9224A0AFD25
:1056F0005C8B261075ED6779BAABEE8F09DF4C3302
:105700006EBF759E987A6019CEBE6F4DEEF22588F9
:1057100095FC5954D860142FD5AC0636ACBF97F51C
:105720001D56273A49A130DE82F8D21C2D2ABD2B06
:10573000FBD212C5091CC1E16DC84FA26DB42D4842
:1057400017D0D5B296A900568E0AB3B3D6C8FB506F
:105750007BC160DC3F7287236C380D47432BD2C47A
:1057600015681A4D67884FC31895EB287C30189F31
:105770005B3585CA851BFAE09F9FC55864D42AA172
:10578000B39401C8F6234D4479FD11C9B23F578443
:10579000FA3814C5442E0DDE5EC1136C726D44469A
:1057A000630FABA1F26186CFEE3D9BDD0FDF3DCDF8
:1057B0007EEAA546756426B34240F0457774EE1B39
:1057C0008D83221FF4C78EC02C97D217BA2C1DFED2
:1057D0005E325E5422F627A8EF6260505EC06741D9
:1057E000D4A9572072EB82889ED694A8FF8B24EF11
:1057F00077D6FBC6A8EB910A8DE81E1E907B644409
:10580000128CD44B47B574CC529E7E2530A17B5769
:10581000437321E8F188C3A61744015AA32BADD7DF
:10582000C435D5D5246C1DC8027622783E8AF70689
:10583000CB62CB13D49D018B59D1D3E85A9E2CE572
:105840007801478B3D7F1FF1E72D73E12CB59785DC
:10585000BB9D8CF843E4DE69A1A0A6DC7135C114C0
:10586000BBE3D4AE662DB254434B0ECD756895DBC9
:10587000D9382554774AAC5460114024DD2A80B9C8
:1058800050BAC0A59E37FA78046B0CC71FBF1FDC47
:105890009F8E6B474EFAFA226947C34595E3C200D3
:1058A0009B256CE1C8A103B86DBF9878B2DEE09685
:1058B00063E92DEA2728380FC87EC0143D2E1B222D
:1058C000C21C57E3F8257920FB923917E13BA0066B
:1058D00067800E7D96581EDD4E341A5BBEAE4A526E
:1058E00078300B11F7E369BB9EB9DA52CDF26DED5A
:1058F000DAC3E6D6681BF400CF3BFC8176209E60BD
:10590000BAC0EA28D235F5ECF4FA618638899C866B
:1059100000F364618B8B1C8330AB1B4E0FE4FAA445
:10592000189909F15058BA62BFD4E11EB485DCD988
:1059300047A144DFE780B636995F34F53083D971EB
:10594000C12EE4CF48E1AC16F1B91B01F736E33ABA
:1059500050E4E01B46FF195AC6C76098FCF5596F22
:10596000081EAE631EA661642F61DFF97A22BC7245
:10597000CFFAF037233800DC2F38FE485F9047C954
:105980002D6E6F1721F42D82EF26FBC831C72D191C
:1059900026155DA987929C35873E0E8FF4E6E9E9CE
:1059A000E91D97BFBFA9C962B2E5297DB4194F248B
:1059B000843047E639D21E22143A9955DAE4A29689
:1059C00074E1991EADDF721B0381D145244CC2AB3B
:1059D000DF67BC3BCE5B5E4C5AD92112539A52B85A
:1059E00044D01D14383343374FCC50B9EA43081B19
:1059F0002D1C7212AE60ACC19F7E75A63F6BEA7A19
:105A00003D87BACE6EDADAFCF84B8B4EE44970E58E
:105A100070A04CE5A4DD7B75516BA13F28D6C0EB8F
:105A2000FDBE84BB8F8013F565DAEE11EC9B440656
:105A300088FF70EEDF7E0CD63F96296584D1ABCC13
:105A40006ABE916A1CC881668652076E9A09D9A5FA
:105A50009A0E98C803609255825BC8FBECE107453B
:105A6000DF3830E0E912F7F42C884227DA1E438051
:105A700008425F72CDF7AFBD8D52A7CC60E89DC5DF
:105A8000A0D6D617D49E118964794B855D4905F659
:105A9000D16FB9F7B635E4DD7A61457CE1268496AD
:105AA00080884CD834927A5671F9F16D6A1DDEB057
:105AB000F97BFD4567D1FA9F25823941DA84FCF4F0
:105AC000251BDCA9BB2F916C35B16DDE40F2BF2BDD
:105AD0006FFAC32BF5AF6BA502152F8DFC9C19F443
:105AE000D42C88E75F7D01FB3459E1F3AA3F93553D
:105AF000063F8B76B4789D42EFB92D4B95A09D4E15
:105B00007C7C74808CAC226C6025AF46837F44BC67
:105B100095526AE9E1D9545EB4D24C538922536F4D
:105B20006B4FF3363518AD0A9E9ED7C3BB6E5858DF
:105B300059DC368E8F3B38396C878C916BC70C02E1
:105B4000D40E67D29C8E0EF0FE2F715C40530DE197
:105B50003B07CE9DDA3122019FE96A0D901A65500C
:105B60003F07549D8B915647ACF3A7C8452BD245B0
:105B70002A06B73EBC7FC1D798C3A25A65CA8B0418
:105B8000A9F1D0528A2DE097439FA5BA3D3159C360
:105B90007560882C26C2E1EBACBB77B13E2A6F075B
:105BA000C70183FF4A730970ED9EE48CEEEFC34694
:105BB000AFE75C420E3FFEA19D6A6DB924F9B9FEC4
:105BC000756F7C90983D8434F6428B896523AC7068
:105BD0008A93CECD89B5A0CE737F4C8EC774829147
:105BE00035804EC3E24FBB2DF0C251919AFE5EDF6D
:105BF000F6C5DEA4C31121BF3EA1DE1810BBE31021
:105C000010CA7D6D83DA0266DE3FD8659F0A653B68
:105C10003E46F1BFBB42409AA1B976FB5F2844C51E
:105C200030541448D45E6772A7D539D8832D33AE6B
:105C30008A29A3E10C9CD4D423CAE4984ECA45AD6A
:105C4000AEC25DEF094A25F8D59F2EB17D81EBE408
:105C50009392EB240E70AF89CF87D51365E9B68C8C
:105C60002EC2C15ACCE4E18DC1401AE23B11D49856
:105C7000A97E66463926339E0B8FDA1E3C1682F6C5
:105C80008ABAFDD4A2B4A1974DF25E8A5DCAE15FE3
:105C9000CD05F95D59A3AFA013524E544866A962D1
:105CA0008C82311D679C3E20AFBF434149695E4AEB
:105CB000C6DE8DED1E0689DD9AAB1794D1B9386921
:105CC000875CF1B2657708BDCD66FBFE208FA1D160
:105CD00052E884FDCEF8533F40446C2BB1A787F5C2
:105CE00000893ECF6D25896A09A6E93FA3F7D753FE
:105CF000983A4B379D2229FA8D2902C33D789A6044
:105D0000F18286AD795AA78A829A1979EE0BDB0463
:105D10004887DEE2B36DB5B73163A5133928DB459B
:105D2000B35E7A65037AC1C39BA986E895DFE8BCB8
:105D3000BE8A88FD725CB1DE90528B9BD61C128E9F
:105D40000322B394D1EC089EFF251B2AF534CB58CF
:105D5000493C178B878D2E37F02A1D68061AC76BB2
:105D6000D6E7F86A8CEF1BAA0F3A60EA849C1C27DE
:105D70000FC39C91EBB44FCF885017EA7BB2296ECA
:105D8000474BBC82D7393D752CBE8A8F4F76DD4498
:105D90006FDD9764D9608177A2E8434C5EF1187E8D
:105DA0005B66CBEDD495A258E9118D25B1575E9273
:105DB00001D2BDE9E09D6B8C94ECE1215B2E514E4C
:105DC00057945EDCFE34A16BC9FD9D3AC3FF3ADCFB
:105DD000B81B9AC40D2D4FD498A402F9F54813723C
:105DE0003A9E157F2950E27A6EEB77904892C68EE4
:105DF000037A7BEF22AC8B781ADB4F54F30FA3BBF3
:105E0000A268AC4974897CDFF9DEFFD39481B103C9
:105E1000753B5507FE8465AC6653424809D6974FDB
:105E200009C1475980F3293FA8BDCFD322C14CDF18
:105E3000FB675D8E90BC1BCEA6F9EAAA2989C146F4
:105E40000437A021A56CA1C0AE268A6A245ADAAF15
:105E500097FE8668A1EBB3A266EB8CA3A4FFA9F61C
:105E6000D4F4FB4C98017C2B8881956AE5DEEDC863
:105E70008748F9BD2670CF635DCE6318049A040D80
:105E800078C3BD9DADF8F97E3B659510E85D398C12
:105E90003E3138DFB9CA65752C08BCE7D7CAAAED10
:105EA000A52E98809EECBA032A8D742A4002F090A9
:105EB000DAE61137FC1E87CE3923C44A02F6B94808
:105EC00052790E0E1E2E29C38CE50679DA75BEF3C3
:105ED0003E30147CA215C187679E194E464707CDF8
:105EE000AC8E4B756D122CB4CAB6C35B384E18FC21
:105EF0007A43F6A841662A345F9C593BF863D6760C
:105F0000F41C0E6DBB4A414E5AC82485E7C49F302D
:105F10008AF8F3C8B8FC7C561466A881BC5C79206A
:105F2000CAE5212BB3C9F08574A33AA44738CC4EF7
:105F300071797873E09E42344D6B0FE3E23FA0111C
:105F4000013B46681116B04C4415897B55044960E5
:105F500073EEA5428FF6B65A828C13249E7E59208A
:105F6000227ACD9926B0CEB7C1CC44B5D83B8E9B12
:105F70003990E88AD139545851198D7E0E513AA77B
:105F80002B9F5DA6EF0F09A04206DC60A349EC8BB6
:105F900089E48D8F87AD5839761E3E50D7C0C5E253
:105FA000FFD66C831B0301E09F8E4FA3DD13518E40
:105FB0004A39EE17AF0AED2A9FF4432D0B7010F506
:105FC000E89B941E21180CAEF10310A2B3BF2CCF96
:105FD000CE656F88E97E641BECED1F67DD3FDADB81
:105FE0000F222873797B47BB5B2626A3FF0E37D988
:105FF000294814AC811D88C2E65BF9CDB7995C9540
:00000001FF
